:100000000C9400010C941D010C941D010C941D0115
:100010000C941D010C941D010C941D010C941D01E8
:100020000C941D010C941D010C941D010C941D01D8
:100030000C941D010C941D010C941D010C941D01C8
:100040000C941D010C941D010C941D010C941D01B8
:100050000C941D01B409AA098F0980099A0977092E
:100060006A09730966093D0D1E0D070D4C0A4C0AFD
:100070004C0A4C0A4C0A4C0A4C0A4C0A4C0A4C0AD0
:100080004C0A4C0A4C0A4C0A4C0A4C0A4C0A4C0AC0
:100090004C0A4C0A4C0A4C0A4C0A4C0A4C0A4C0AB0
:1000A0004C0A4C0A4C0A4C0A4C0A4C0A4C0A4C0AA0
:1000B0004C0A4C0A4C0AFE0C980D510DCF0CAB0C9F
:1000C000060EE70D1E0EEC0CA80DA10DBB0DBB0D11
:1000D000B60B4D0C420C370C2D0C1D0C100CC70B25
:1000E0004C0A4C0A4C0A4C0A4C0A4C0A4C0A4C0A60
:1000F0004C0A4C0A4C0A4C0A4C0A4C0A4C0A4C0A50
:100100004C0A4C0A4C0A4C0ABC0BA00C910C5D0C1E
:10011000530C4C0A4C0A4C0AAC0BA20B4C0A4C0A6E
:100120004C0A4C0A4C0A4C0A4C0A4C0A4C0A4C0A1F
:100130004C0A4C0A4C0A4C0A4C0A4C0A4C0A4C0A0F
:100140004C0A4C0A4C0A4C0A4C0A4C0A4C0A4C0AFF
:100150004C0A4C0A4C0A930B710B5E0B1E0B4C0A9B
:100160004C0A4C0A4C0A4C0A4C0A4C0A4C0A4C0ADF
:100170004C0A4C0A4C0A4C0A4C0A4C0A4C0A4C0ACF
:100180004C0A4C0A4C0A4C0A4C0A4C0A4C0A4C0ABF
:100190004C0A4C0A4C0A4C0A4C0A4C0A4C0A4C0AAF
:1001A0004C0A4C0A4C0AE80AC30A4C0A4C0A4C0A8C
:1001B0004C0A4C0A4C0A4C0A4C0A4C0A4C0A4C0A8F
:1001C0004C0A4C0A4C0A4C0A4C0A4C0A4C0A4C0A7F
:1001D0004C0A4C0A4C0A4C0A4C0A4C0A4C0A4C0A6F
:1001E0004C0A4C0A4C0A4C0A4C0A4C0A4C0A4C0A5F
:1001F0004C0A4C0A4C0A9B0A840A6579312E30005D
:1002000011241FBECFE5D8E0DEBFCDBF10E0A0E6D1
:10021000B0E0E0EDFDE102C005900D92A636B10719
:10022000D9F727E0A6E6B0E001C01D92AA37B207D1
:10023000E1F70E94E6090C94E60E0C94000091ECA4
:1002400096B94431510570F04832510508F049C063
:1002500092EC9093740708C0403491E0590708F479
:100260004FC096EC9093740792E09EBD806687B96C
:1002700041505109AF9A349BFECF329A10927907C0
:10028000109278076115710549F11DBC1CBC809165
:10029000740786B9349BFECF8091760790917707DB
:1002A0009C012F5F3F4F309377072093760725B14E
:1002B000FC01E759FF4F2083329A8CB590E08417F8
:1002C0009507D8F3809178079091790701969093DC
:1002D00079078093780786179707B8F216B8AF9812
:1002E00008954035510540F0403A510508F0B4CF2B
:1002F00094EC90937407B8CF93EC90937407B4CFB9
:1003000095EC90937407B0CF0F931F93CF93DF9327
:10031000282F217030E0220F331F122F1160F82F89
:10032000F270F160847090E095958795D82FD16038
:10033000425082E08EBDAF9A1092790710927807F2
:100340006115710509F487C0C3E0E0E154E10CE1F7
:100350001CBCC8BBE2BB52BBE2BB52BBD8BBE2BBBE
:1003600052BBF8BBE2BB52BB18BBE2BB52BB52BB99
:10037000E2BBE2BB52BBE2BB52BBE2BB52BB86B3A9
:10038000817080937307E2BB52BB86B39091730771
:10039000990F8170982B90937307E2BB52BB86B381
:1003A00090917307990F8170982B90937307E2BB1C
:1003B00052BB86B390917307990F8170982B9093DD
:1003C0007307E2BB52BB36B390917307990F31703C
:1003D000932B90937307E2BB52BB36B39091730794
:1003E000990F3170932B90937307E2BB52BB36B3D6
:1003F00090917307990F3170932B90937307E2BB21
:1004000052BB36B390917307990F3170932B909331
:10041000730702BB9CB59417E8F38091760790911F
:1004200077079C012F5F3F4F309377072093760724
:1004300087599F4F20917307DC012C938091780797
:1004400090917907019690937907809378078617A2
:10045000970708F47DCFAF98DF91CF911F910F914F
:1004600008950F931F93CF93DF93282F217030E0CF
:10047000220F331F122F1160F82FF270F160847079
:1004800090E095958795D82FD160425082E08EBD3F
:10049000AF9A10927907109278076115710509F4E7
:1004A0008AC0C3E0E0E154E10CE11CBCC8BBE2BB84
:1004B00052BBE2BB52BBD8BBE2BB52BBF8BBE2BBF8
:1004C00052BB18BBE2BB52BB52BBE2BBE2BB52BB4E
:1004D000E2BB52BBE2BB52BB86B381708093730711
:1004E000E2BB52BB86B390917307990F8170982B32
:1004F00090937307E2BB52BB86B390917307990F39
:100500008170982B90937307E2BB52BB86B3909196
:100510007307990F8170982B90937307E2BB52BBBE
:1005200036B390917307990F3170932B90937307A3
:10053000E2BB52BB36B390917307990F3170932B86
:1005400090937307E2BB52BB36B390917307990F38
:100550003170932B90937307E2BB52BB36B39091EB
:100560007307990F3170932B9093730702BB9CB55F
:100570009417E8F300000000000080917607909146
:1005800077079C012F5F3F4F3093770720937607C3
:1005900087599F4F20917307DC012C938091780736
:1005A0009091790701969093790780937807861741
:1005B000970708F47ACFAF98DF91CF911F910F91F1
:1005C0000895CF93DF9322E02EBD660F6250AF9A5D
:1005D0001092790710927807009709F4FAC0F3E0B7
:1005E000E0E174E1B1E0ACE11CBCF8BBE2BB72BB82
:1005F000E2BB72BBB8BBE2BB72BBE2BB72BBE2BB8D
:1006000072BB72BBE2BBE2BB72BBE2BB72BBE2BBC2
:1006100072BB26B3217020937307E2BB72BB36B363
:1006200020917307220F3170232B20937307E2BBB5
:1006300072BB36B320917307220F3170232B2093A6
:100640007307E2BB72BB36B320917307220F317080
:10065000232B20937307E2BB72BB36B32091730741
:10066000220F3170232B20937307E2BB72BB36B38A
:1006700020917307220F3170232B20937307E2BB65
:1006800072BB36B320917307220F3170232B209356
:100690007307E2BB72BB36B320917307220F317030
:1006A000232B20937307A2BB209176073091770705
:1006B000A9014F5F5F4F5093770740937607E90199
:1006C000C759DF4F409173074883F8BBE2BB72BB49
:1006D000E2BB72BBB8BBE2BB72BBE2BB72BBF8BB96
:1006E000E2BB72BB72BBE2BBE2BB72BBE2BB72BBE2
:1006F000E2BB72BB26B3217020937307E2BB72BBCF
:1007000036B320917307220F3170232B2093730788
:10071000E2BB72BB36B320917307220F3170232BDB
:1007200020937307E2BB72BB36B320917307220F8D
:100730003170232B20937307E2BB72BB36B3209139
:100740007307220F3170232B20937307E2BB72BB18
:1007500036B320917307220F3170232B2093730738
:10076000E2BB72BB36B320917307220F3170232B8B
:1007700020937307E2BB72BB36B320917307220F3D
:100780003170232B20937307A2BB2CB52617E8F3F7
:100790002091760730917707A9014F5F5F4F509303
:1007A000770740937607E901C759DF4F40917307F8
:1007B00048830000000020917807309179072F5F6F
:1007C0003F4F30937907209378072817390708F4AB
:1007D0000BCFAF98DF91CF910895FF920F931F93A6
:1007E000CF93DF93282F217030E0220F331F122F79
:1007F0001160C82FC270C160847090E09595879594
:10080000282F2160F22E4250510982E08EBDAF9A0E
:1008100010927907109278076115710509F4DBC011
:1008200003E0A0E1B4E1DCE11DBC1CBC08BBA2BB41
:10083000A2BBB2BBB2BBA2BBA2BBB2BBF8BAA2BB4B
:10084000A2BBB2BBC8BBA2BBA2BBB2BB18BBA2BB04
:10085000A2BBB2BBB2BBB2BBB2BBB2BBB2BBA2BB50
:10086000A2BBB2BBB2BBB2BBB2BBB2BBB2BBA2BB40
:10087000A2BBB2BBB2BBA2BBA2BBB2BB86B38170F0
:1008800080937307A2BBA2BBB2BB96B380917307E0
:10089000880F9170892B80937307A2BBA2BBB2BB58
:1008A00096B380917307880F9170892B809373079B
:1008B000A2BBA2BBB2BB96B380917307880F9170A5
:1008C000892B80937307A2BBA2BBB2BB96B3809166
:1008D0007307880F9170892B80937307A2BBA2BB0B
:1008E000B2BB96B380917307880F9170892B809368
:1008F0007307A2BBA2BBB2BB86B390917307990FDB
:100900008170982B90937307A2BBA2BBB2BB86B336
:1009100090917307990F8170982B90937307A2BBE6
:10092000A2BBB2BB86B3817080937407A2BBA2BB8B
:10093000B2BB86B390917407990F8170982B9093F6
:100940007407A2BBA2BBB2BB86B390917407990F88
:100950008170982B90937407A2BBA2BBB2BB86B3E5
:1009600090917407990F8170982B90937407D2BB64
:10097000809164008230B0F1809176079091770782
:10098000FC01E759FF4F209174072295207F2083B7
:1009900001969C012F5F3F4F309377072093760796
:1009A000FC01E759FF4F2091730720838CB59DB55B
:1009B00084179507D8F300000000000080917807A5
:1009C000909179070196909379078093780786171D
:1009D000970708F429CFAF98DF91CF911F910F911E
:1009E000FF9008958091760790917707D2CF0F936B
:1009F0001F93CF93DF9361507048660F771F22E0FB
:100A00002EBDAF9A1092790710927807009709F4DB
:100A1000A3C1B3E0E0E1F4E1A1E00CE11DBC1CBC2A
:100A2000B8BBE2BBE2BBF2BBF2BBE2BBE2BBF2BBD8
:100A3000A8BBE2BBE2BBF2BBA8BBE2BBE2BBF2BB22
:100A4000A8BBE2BBE2BBF2BBF2BBF2BBF2BBF2BBA8
:100A5000F2BBE2BBE2BBF2BBF2BBF2BBF2BBF2BB4E
:100A6000F2BBE2BBE2BBF2BBF2BBE2BBE2BBF2BB5E
:100A700026B3217020937307E2BBE2BBF2BB36B30F
:100A800020917307220F3170232B20937307E2BB51
:100A9000E2BBF2BB36B320917307220F3170232BD8
:100AA00020937307E2BBE2BBF2BB36B3209173071E
:100AB000220F3170232B20937307E2BBE2BBF2BB02
:100AC00036B320917307220F3170232B20937307C5
:100AD000E2BBE2BBF2BB36B320917307220F317049
:100AE000232B20937307E2BBE2BBF2BB36B320910A
:100AF0007307220F3170232B20937307E2BBE2BBF5
:100B0000F2BB36B320917307220F3170232B209351
:100B10007307E2BBE2BBF2BB26B3217020937407DC
:100B2000E2BBE2BBF2BB36B320917407220F3170F7
:100B3000232B20937407E2BBE2BBF2BB36B32091B8
:100B40007407220F3170232B20937407E2BBE2BBA2
:100B5000F2BB36B320917407220F3170232B209300
:100B6000740702BB20916400223008F4FBC020917E
:100B7000760730917707A90147595F4F10917407A5
:100B80001295107FEA0118832F5F3F4FA9014F5F35
:100B90005F4F509377074093760727593F4F409117
:100BA0007307E9014883B8BBE2BBE2BBF2BBF2BB0F
:100BB000E2BBE2BBF2BBA8BBE2BBE2BBF2BBA8BBA1
:100BC000E2BBE2BBF2BBB8BBE2BBE2BBF2BBF2BB37
:100BD000F2BBF2BBF2BBF2BBE2BBE2BBF2BBF2BBCD
:100BE000F2BBF2BBF2BBF2BBE2BBE2BBF2BBF2BBBD
:100BF000E2BBE2BBF2BB26B3217020937307E2BBDA
:100C0000E2BBF2BB36B320917307220F3170232B66
:100C100020937307E2BBE2BBF2BB36B320917307AC
:100C2000220F3170232B20937307E2BBE2BBF2BB90
:100C300036B320917307220F3170232B2093730753
:100C4000E2BBE2BBF2BB36B320917307220F3170D7
:100C5000232B20937307E2BBE2BBF2BB36B3209198
:100C60007307220F3170232B20937307E2BBE2BB83
:100C7000F2BB36B320917307220F3170232B2093E0
:100C80007307E2BBE2BBF2BB36B320917307220FBE
:100C90003170232B20937307E2BBE2BBF2BB26B378
:100CA000217020937407E2BBE2BBF2BB36B3209104
:100CB0007407220F3170232B20937407E2BBE2BB31
:100CC000F2BB36B320917407220F3170232B20938F
:100CD0007407E2BBE2BBF2BB36B320917407220F6C
:100CE0003170232B2093740702BB209164002230C3
:100CF00008F43DC02091760730917707A901475944
:100D00005F4F109174071295107FEA0118832F5FCF
:100D10003F4FA9014F5F5F4F50937707409376078E
:100D200027593F4F40917307E90148832CB53DB5E2
:100D300026173707D8F3000000000000209178073D
:100D4000309179072F5F3F4F3093790720937807D1
:100D50002817390708F462CEAF98DF91CF911F9121
:100D60000F91089520917607309177070FCF20914A
:100D7000760730917707CDCF33E038BB90E192BB57
:100D800092BB24E122BB22BB92BB92BB22BB82FF5F
:100D9000B7C038BB90E192BB92BB94E192BB81FF9C
:100DA000ACC093E098BB90E192BB92BB94E192BB44
:100DB00080FFA0C083E088BB80E182BB82BB94E15E
:100DC00092BB82BB82E08EBD1DBC1CBC90916300B7
:100DD0008CB58917E8F394E192BB92BB80E182BBAA
:100DE00082BB92BB92BB82BB82BB92BB26B32170FB
:100DF0002093730782BB82BB92BB36B320917307EB
:100E0000220F3170232B2093730782BB82BB92BBCE
:100E100036B320917307220F3170232B2093730771
:100E200082BB82BB92BB36B320917307220F317015
:100E3000232B2093730782BB82BB92BB26B3217006
:100E40002093740782BB82BB92BB36B32091740798
:100E5000220F3170232B2093740782BB82BB92BB7D
:100E600036B320917407220F3170232B209374071F
:100E700082BB82BB92BB36B320917407220F3170C4
:100E8000232B2093740782BB82BB92BB36B3209185
:100E90007407220F3170232B2093740782BB82BB0F
:100EA00092BB36B320917407220F3170232B20930D
:100EB000740782BB82BB92BB36B320917407220FAA
:100EC0003170232B2093740782BB82BB92BB96B3F5
:100ED00080917407880F9170892B809374078CE13F
:100EE00082BB8091730790E0982F88272091740728
:100EF000822B089581E088BB5FCF91E098BB53CFF0
:100F000091E098BB47CF282F217030E0220F331F8C
:100F10002160482F42704160847090E095958795DC
:100F2000816093E098BB30E132BB94E192BB32BB6D
:100F300092BB88BB32BB92BB48BB32BB92BB28BBC7
:100F400032BB92BB92BB32BB32BB92BB32BB92BBB9
:100F500032BB92BB86B381708093730732BB92BB66
:100F600026B380917307880F2170822B80937307BB
:100F700032BB92BB26B380917307880F2170822BFE
:100F80008093730732BB92BB26B380917307880F9F
:100F90002170822B8093730732BB92BB26B3809162
:100FA0007307880F2170822B8093730732BB92BB2B
:100FB00026B380917307880F2170822B809373076B
:100FC00032BB92BB26B380917307880F2170822BAE
:100FD0008093730732BB92BB96B380917307880FDF
:100FE0009170892B809373078CE182BB089598E000
:100FF00092BB880F816088BB92BB92BB8CE082BBA6
:1010000082BB23E028BB92BB92BB82BB82BB28BBC6
:1010100092BB92BB82BB82BB28BB92BB92BB82BB02
:1010200082BB80E098E090937907809378071092D4
:101030007307E1E053E048E03CE016C058BB42BB18
:1010400042BB32BB32BB809178079091790796956D
:1010500087959093790780937807209173072F5F86
:10106000209373072C3030F486239723892B31F794
:10107000E8BBE5CF8CE182BB08958823B1F093B340
:101080009823A9F42CB53DB52135334CB0F31DBCE4
:101090001CBC909168009F5F90936800993268F340
:1010A00084E58093690080E008954599EBCF81E065
:1010B0000895482F50E00DC023B330E020953095BF
:1010C00024233523232B49F42CB53DB52135334C4E
:1010D00030F48111F1CF459BF7CF81E008951DBC1D
:1010E0001CBC909168009F5F90936800993288F3D0
:1010F00084E58093690080E008951092680008C03C
:1011000093B3982349F42CB53DB52135334C50F4B5
:101110008111F6CF4599F7CF1DBC1CBC1092680019
:1011200081E008951DBC1CBC909168009F5F909366
:101130006800993268F384E58093690080E008953F
:1011400010926800482F50E00DC023B330E0209586
:10115000309524233523232B49F42CB53DB5213577
:10116000334C50F48111F1CF459BF7CF1DBC1CBC13
:101170001092680081E008951DBC1CBC909168002D
:101180009F5F90936800993268F384E580936900CB
:1011900080E008956091680008C093B3982349F4F3
:1011A0002CB53DB52135334C58F58111F6CF459915
:1011B000F7CF8091760790917707AC014F5F5F4F33
:1011C00050937707409376072CB5FC01E759FF4F02
:1011D00020839C012E5F3F4F309377072093760743
:1011E0007DB5FA01E759FF4F708303969093770717
:1011F00080937607F901E759FF4F608381E00895F6
:101200001DBC1CBC6F5F60936800693270F284E59E
:101210008093690080E0089560916800482F50E055
:101220000DC023B330E02095309524233523232BA4
:1012300049F42CB53DB52135334C58F58111F1CF2A
:10124000459BF7CF8091760790917707AC014F5F70
:101250005F4F50937707409376072CB5FC01E75911
:10126000FF4F20839C012E5F3F4F309377072093E1
:1012700076077DB5FA01E759FF4F70830396909387
:10128000770780937607F901E759FF4F608381E084
:1012900008951DBC1CBC6F5F60936800693270F2DA
:1012A00084E58093690080E00895CF93C82F1DBC2A
:1012B0001CBC109268004091750750E04930510500
:1012C00068F4FA01E65DFF4F0C94C20E809167004E
:1012D0000E943D08809167000E94590884E4809331
:1012E0006900CF910895809167000E94590880910C
:1012F00067000E943D0884E480936900CF910895BF
:1013000085B390916700892B85BB1DBC1CBC2091C7
:10131000620030E08CB59DB582179307D8F395B382
:10132000809167008095892385BB84E48093690060
:10133000CF91089595B3809167008095892385BBEF
:101340001DBC1CBC2091620030E08CB59DB582179D
:101350009307D8F385B390916700892B85BB84E40C
:1013600080936900CF9108951092790710927807C1
:101370008C2F0E94830780917307809374071DBC94
:101380001CBC2CB53DB524313105D8F38C2F0E94FF
:1013900083079091730780917407891748F48091AF
:1013A0006100981728F080916000891708F096CFA7
:1013B00020917807309179072F5F3F4F309379075D
:1013C00020937807283C310598F288CFCF93DF939C
:1013D00000D000D000D0CDB7DEB78FE18ABB1BBAFA
:1013E0008AE087BB80EF84BB8CE981BB83E085BB4F
:1013F00088E18AB910BC8CE089B986EA80BD80E4B6
:1014000088B982E08EBD109277071092760729E6A0
:10141000C22E20E0D22E38E2732E44E4542EEE2465
:10142000E394F12C02E010E0C094D0949701295687
:101430003040590168E0462E79E1672E80917607A9
:10144000909177075F9BFECFFC0101969093770701
:10145000809376072CB1E759FF4F2083789EA00137
:10146000799E500D11242091690030E02417350732
:1014700048F7109268001DBC1CBC20916900509276
:101480006900F0927707E0927607822F90E0FC01E6
:101490003197EA3CF10580F0F3E4F093690083E4CE
:1014A0005D9BFECF8CB980916900843449F0109225
:1014B000770710927607C2CFED5CFF4F0C94C20EF7
:1014C000F0927907E09278078091760790917707FC
:1014D000029768F381E090E05D9BFECFFC01E75945
:1014E000FF4F80818CB980917807909179070196A0
:1014F000909379078093780720917607309177074A
:101500008217930748F3D3CF40916E0050E0542FD9
:10151000442780916D00482B60916C0070E0762F1D
:10152000662780916B00682B80916A000E941F01E2
:1015300080916900B5CF30906A0080916C0090E096
:10154000382F222780916B00282B3C832B8380909F
:101550006D0020916E00309164004B815C81349F5E
:10156000C001359F900D11248930974040F4912C93
:10157000922AC4014497853D934008F465C381E4F1
:10158000809369008DCF90906A0020906C00312C80
:10159000322C222480916B00282A60916D0039E062
:1015A000231637E0330658F786EF860F8B3538F76A
:1015B00070E0892D0E94550940916D00B101892D7F
:1015C0004A3009F45EC30E9431028091690068CFFD
:1015D00080906B00912C982C882480916A00882A36
:1015E00020906C0050916D0040916400842F90E039
:1015F000880F991F889D9001899D300D989D300D11
:1016000011242930374008F0BACF312C352AC101D6
:101610004497853D934008F0B2CF1093770700932D
:10162000760740936A00B10180E00E945509B1013C
:10163000C4010E94F7048091690032CF80906B0052
:10164000912C982C882480916A00882A909279079E
:101650008092780780916C0010927407882309F4B7
:1016600024C34AE650E08150282E312C910125599F
:101670003F4F19019A018C0C9D1CC501820F931FCD
:101680009093770780937607C401820F931F298375
:101690003A834D835E830E94D10E29813A81F901FC
:1016A00081939F014D815E818E2F841B80937407EF
:1016B000E215F30511F780916900F2CE80916B007D
:1016C00090E0982F882720916A00822B90937907C9
:1016D0008093780760916C000E94D90E8091690018
:1016E000DFCE80906B00912C982C882480916A002A
:1016F000882A60916C00C401880F991F8930974037
:1017000008F03DCF86EF860F8B3508F038CF70E0BC
:1017100080E00E94550960916C00C4010E94E102C2
:1017200080916900BDCE60916C0070E0762F6627D5
:1017300080916B00682B80916A000E94F70780916E
:101740006900AECE80916A008111B1C280916B00B8
:101750008BBB80916900A4CE80916A008111C5C2C3
:1017600080916B008ABB809169009ACE80916A005B
:101770008093620084E494CE80916A0087708861CF
:1017800083BF80916B008CBF8091690089CE88E611
:1017900083BD65BC1DBC1CBC8CB59DB5843C99400B
:1017A000D8F315BC1DBC1CBC8CB59DB5843F9140C5
:1017B000D8F380916A00809374071092730765BC18
:1017C0001DBC1CBC8CB59DB5843F9140D8F315BCA5
:1017D0001DBC1CBC8CB59DB5843F9140D8F32091B5
:1017E000740727FD32C0220F20937407809173077E
:1017F0008F5F80937307883010F365BC1DBC1CBCE1
:101800008CB59DB5843F9140D8F315BC1DBC1CBC64
:101810008CB59DB5843F9140D8F38091690040CE4E
:1018200080916A00811132C2109377070093760786
:1018300089B380936A0084E433CE80916A00811179
:1018400060C213BE809169002BCE1DBC1CBC8CB540
:101850009DB5843F9140D8F3C6CF80916A0088231C
:1018600081F38CBF8BE683BF8091690019CE809194
:101870006A00883008F035C287B940BE16B880913A
:1018800069000ECE80916A00E0E18E9FC0011124B4
:10189000836085BB8091690003CE80916A0080934C
:1018A000660084E4FDCD80916A00809361008091A0
:1018B0006B008093600084E4F3CD80916A008F70A8
:1018C000809374071DBC1CBC0E945908882309F42E
:1018D000F2CE809174070E947D08882309F4EBCE34
:1018E000809174070E945908882309F4E4CE8091FE
:1018F0006B009FEF980F90936B00882361F08091AD
:1019000074070E943D08882331F0809174070E947B
:1019100059088111ECCF809169008435C9F584E5BF
:10192000BFCD80916A00853008F0CFC180937507E4
:1019300080916B008295807F8093670084E4B0CDB6
:1019400080916A008770886185BD80916B0083BD3E
:1019500080916900A5CD90916A00892F82958F7042
:10196000809373079F70909374070E94590888238F
:1019700009F4A1CE809173070E947D08882309F4A1
:101980009ACE809174070E945908882309F493CE57
:10199000809174070E94CA088091690081CD90915E
:1019A0006A00892F82958F70809373079F70909340
:1019B00074070E945908882309F47DCE809173072B
:1019C0000E947D08882309F476CE809174070E94D6
:1019D0000C098091690064CD95B380916A00807F85
:1019E000892B85BB109268001DBC1CBC80916A00CD
:1019F0008F700E940C098091690052CD80916A001D
:101A00008B3F08F0BCCD8093630084E449CDAC9A51
:101A10001DBC1CBC809162009CB59817E8F3AC9883
:101A2000109268001DBC1CBC8CB59DB50597E0F3F9
:101A300084E00E94CA088091690032CDF5E0F7B9D0
:101A400040BE16B82091760730917707C9010196FC
:101A5000909377078093760743B388B1F901E759EC
:101A6000FF4F807290E09595879595958795477083
:101A7000482B40838091690013CD45E050E06AEF28
:101A800071E08AE690E00E94C80E809176079091FE
:101A90007707059690937707809376078091690082
:101AA000FFCC80916A000E94BC06909379078093D6
:101AB000780780916A000E94BC06209178073091D7
:101AC0007907280F391F3093790720937807809181
:101AD0006A000E94BC062091780730917907280F90
:101AE000391F309379072093780780916A000E940C
:101AF000BC062091780730917907280F391F369559
:101B0000279536952795309379072093780780910C
:101B1000760790917707FC01E759FF4F20830296E3
:101B20009093770780937607318380916900B8CCD2
:101B300080916A00833008F022CD8093640084E4B1
:101B4000AFCC95B380916A00807F8095892349CF7F
:101B500095B380916A00807F8095892385BB109220
:101B600068001DBC1CBC80916A008F700E94CA086E
:101B70008091690095CC90916A00892F807F809335
:101B800073079F709093740790916600992309F4EE
:101B9000BEC095B3982B95BB1DBC1CBC8091620048
:101BA0009CB59817E8F395B38091730780958923C6
:101BB00085BB109268001DBC1CBC8CB59DB50597FB
:101BC000E0F380917407243309F013CFCFCF9091C5
:101BD0006A00892F82958F70809373079F7090930E
:101BE00074070E943D08882309F465CD809173072E
:101BF0000E94A008882309F45ECD809174070E949A
:101C00003D088111E2CE809169004ACC90916A0032
:101C1000892F82958F70809373079F7090937407BC
:101C20000E943D08882309F446CD809173070E94E5
:101C3000A0088111ADCE8091690032CC95B380911E
:101C40006A00807F892B8ACFB401832D0E945509B9
:101C50002091760730917707C90101969093770715
:101C600080937607F901E759FF4F809164008083E4
:101C7000A4016B817C81832D0E94ED03809169001A
:101C80000FCC0E948401809169000ACC813009F454
:101C900064C0823009F458C0833039F41093770758
:101CA0000093760780B380936A0084E4F9CB813097
:101CB00009F462C0823009F459C08330B1F78091D1
:101CC0006B0082BB80916900EBCB893008F057CC68
:101CD0008093750780916B008F708093670084E418
:101CE000DFCB10BE80916900DBCB813039F18230CF
:101CF000F9F08330D1F680916B0081BB809169004F
:101D0000CFCB8CBF89E683BF80916900C9CB95B3E7
:101D10008095892385BB1DBC1CBC809162009CB54D
:101D20009817E8F385B390917307892B85BB41CF52
:101D300080916B0084BB80916900B2CB80916B0075
:101D400087BB80916900ACCB10937707009376072F
:101D500083B380936A0084E4A3CB10937707009346
:101D6000760786B380936A0084E49ACB80916B00F7
:101D700085BB8091690094CB80916B0088BB80917A
:101D800069008ECBEE0FFF1F0590F491E02D0994B2
:101D9000FB01DC0102C005900D9241505040D8F784
:101DA0000895E199FECF9FBB8EBBE09A99278DB332
:101DB0000895262FE199FECF9FBB8EBB2DBB0FB69A
:101DC000F894E29AE19A0FBE01960895F894FFCF35
:061DD000837D0DC8010037
:00000001FF
